:020000040000FA
:040000008A010E283B
:0800080009000C1C05280C1076
:1000100005110C1C09280C10051508009B20203028
:1000200090008E018F011014052005200520851FEA
:100030002128A2182128A2140C1E1C28FA3099008D
:100040000511851B2B28A21C2B28A2100C1E26286C
:10005000FC3099000515051F342822193428221573
:100060000C1E3028F8309900051B3928221D39282C
:1000700022118C1E1728811A7420981C41281812EE
:100080001816181D44281A088C1E3B281A080C1E26
:1000900047289900A0002008F83A0319602020089A
:1000A000FA3A031964202008FB3A03196B20200850
:1000B000FC3A03196F202008CF3A031977203B2818
:1000C000051481018D200800851405148101A1010A
:1000D000051122140800851405112214080085104A
:1000E00005100515221008000510810108008C1E5E
:1000F00077281A080C1E7A2899001F39A000A3013E
:100100002018A317A01823172019A316A019231627
:10011000201AA315230886000800A10A2108013A25
:10012000031905112108033A031905152108183A86
:100130000319A101080007309F00831603139F01D4
:10014000073099002430980086308100C030850047
:10015000063086008C1483120313A001A101A201B2
:1001600000308500003086000515A00105108510BF
:100170009801900100009030980000308B0008003A
:02400E00101F81
:104200002834633429343234303430343634203472
:104210004434743472346F346E34693463347334B8
:104220007734773477342E346434743472346F34A2
:104230006E346934633473342E346E3465347434BC
:00000001FF
